:100000000C94A1000C940E290C9439290C946429A9
:100010000C94CB000C94CB000C94CB000C94CB0034
:100020000C94CB000C94CB000C94CB000C94CB0024
:100030000C94CB000C94CB000C94CB000C94CB0014
:100040000C94CB000C94CB000C942E270C94CB007A
:100050000C9444250C947A250C94CB000C94CB0082
:100060000C94CB000C94CB000C94CB000C94CB00E4
:100070000C94CB000C94CB000C94CB000C94CB00D4
:100080000C94CB000C94CB000C94CB00D81FBC1F5D
:10009000DB1FBF1FC21FC51FC81FCB1FCF1FD31F12
:1000A0004128442837283B285B285B2848284C28CF
:1000B00052285628D729DC29E129EB29192A192A9F
:1000C000F529FD29052A0F2A000000010200090A6E
:1000D000000000000403080700000000000000000A
:1000E0000000000000000000010204081020408011
:1000F0000102040810204080010204081020408002
:1001000001020408102040800202020202020202E0
:1001100004040404040404040303030303030303A7
:100120000101010101010101000022002500280058
:100130002B0000002100240027002A00C1055023C5
:10014000AE2511241FBECFEFD0E4DEBFCDBF11E03E
:10015000A0E0B1E0E6E4F9E500E00BBF02C00790E3
:100160000D92AE34B107D9F729E3AEE4B1E001C096
:100170001D92A833B207E1F710E0C1EAD0E004C055
:100180002197FE010E94DD2ACE39D107C9F70E94CE
:10019000DC250C94A12C0C9400001F93CF93DF93CB
:1001A000EC01162F0E94832C181739F0612FCE0115
:1001B000DF91CF911F910C948B2CDF91CF911F91E8
:1001C00008950C94832CDC01ED91FC910190F08159
:1001D000E02D099461E08CE00C94982860E08CE0BC
:1001E0000C94982861E08DE00C94982860E08DE0F4
:1001F0000C9498280F931F93CF93DF938C01009753
:1002000011F0EC0102C0C1E0D0E01C161D060CF597
:1002100061E08CE00E94982860E08DE00E949828C0
:1002200064E670E080E090E00E94A92760E08CE046
:100230000E94982861E08DE00E94982864E670E0B2
:1002400080E090E00E94A92701151105F1F22197A5
:10025000DCCF60E08CE00E94982860E08DE0DF91C8
:10026000CF911F910F910C9498280F931F93CF93C8
:10027000DF938C01009711F0EC0102C0C1E0D0E0E7
:1002800061E08DE00E94982860E08DE01C161D065C
:10029000BCF40E94982864E670E080E090E00E9440
:1002A000A92761E08DE00E94982864E670E080E074
:1002B00090E00E94A9270115110531F32197E4CFA1
:1002C000DF91CF911F910F910C9498280F931F935A
:1002D000CF93DF938C01009711F0EC0102C0C1E0D5
:1002E000D0E060E08CE01C161D06BCF40E9498284B
:1002F00064E670E080E090E00E94A92761E08CE075
:100300000E94982864E670E080E090E00E94A927AF
:100310000115110531F32197E4CFDF91CF911F91A2
:100320000F910C94982880914E0190914F01A091CB
:100330005001B09151010196A11DB11D80934E0154
:1003400090934F01A0935001B0935101409104014B
:1003500050910501609106017091070148175907F6
:100360006A077B0720F510924E0110924F01109200
:10037000500110925101609153018091090186173B
:1003800010F081E005C080910801681718F08FEF28
:100390008093520180915201680F6093530170E085
:1003A0008CE00E94B02960E08DE00C9498280895BC
:1003B00080914E0190914F01A0915001B091510157
:1003C0000196A11DB11D80934E0190934F01A09302
:1003D0005001B09351014091040150910501609189
:1003E000060170910701481759076A077B0720F536
:1003F00010924E0110924F01109250011092510133
:100400006091530180910901861710F081E005C0C9
:1004100080910801681718F08FEF80935201809146
:100420005201680F6093530170E08DE00E94B02983
:1004300060E08CE00C949828089560EC70E08EE801
:1004400098E30E94E30066E070E08EE898E30E9483
:10045000E3006091613870E08EE898E30E94E30069
:1004600060EC70E08EE898E30C94E30060EC70E0E0
:100470008EE898E30E94E30067E070E08EE898E37E
:100480000E94E3006091190170E08EE898E30E94F9
:10049000E30060EC70E08EE898E30C94E30060EC1D
:1004A00070E08EE898E30E94E3006FE070E08EE871
:1004B00098E30E94E30061E070E08EE898E30E9418
:1004C000E30060EC70E08EE898E30C94E30060ECED
:1004D00070E08EE898E30E94E3006EE070E08EE842
:1004E00098E30E94E30080915F38882319F061E06F
:1004F00070E002C060E070E08EE898E30E94E300E4
:1005000060EC70E08EE898E30C94E30060EC70E03F
:100510008EE898E30E94E30068E070E08EE898E3DC
:100520000E94E30066E470E08EE898E30E94E30036
:1005300060EC70E08EE898E30C94E30060EC70E00F
:100540008EE898E30E94E30060E570E08EE898E3AF
:100550000E94E30061E070E08EE898E30E94E3000F
:100560006AE070E08EE898E30E94E30060EC70E0DF
:100570008EE898E30C94E30080916138882341F081
:1005800060916A3870916B388CE698E30C941D2169
:10059000089580916138882341F060911C01709129
:1005A0001D018CE698E30C94F9210895809161383F
:1005B0008823E1F080915E38843A51F460911A0109
:1005C00070911B0140E050E08CE698E30E943123DB
:1005D00080915E38893A51F460911A0170911B0143
:1005E00041E050E08CE698E30C943123089580912B
:1005F0006138882361F08CE698E30E94AB1F60931A
:100600006638709367388093683890936938089596
:1006100080916138882371F0409166385091673835
:1006200060916838709169388CE698E30E9459218E
:100630000C94F702089580916138882361F08CE66C
:1006400098E30E947B1F60936238709363388093B5
:10065000643890936538089580916138882371F0EB
:100660004091623850916338609164387091653878
:100670008CE698E30E94CE200C941B030895809191
:100680006138882321F08CE698E30C94E01F80E029
:100690000895C8E3DFE06FEFCE010E94CD00219600
:1006A000C11580E1D807B9F70E94F2000E94EE0060
:1006B000FBCF83ED9FE00E94E10091E0833709F0DA
:1006C00090E0892F089588E39FE00E94E10091E087
:1006D000833009F090E0892F089589E39FE00E941C
:1006E000E100982F80935E3881E0943A21F0993AA6
:1006F00011F080E0089508958AE39FE00E94E100F0
:1007000080935D389FEF980F81E09E3F08F080E076
:100710000895BF92CF92DF92EF92FF920F931F93B3
:10072000CF93DF938BE090E00E940D267C018C013B
:10073000C8E3DFE0CE010E94E100F80181938F0160
:100740002196C334FFE0DF07A9F76BE070E0C70133
:100750000E94571EB82EC92E082F192FDD24D394BE
:10076000CE010E94E100F80191918F018913D12CF3
:100770002196C335FFE0DF0799F78B2D9C2D0E9452
:10078000A526C7010E94A5268D2DDF91CF911F912F
:100790000F91FF90EF90DF90CF90BF9008958FED75
:1007A0009FE00E94E10091E0833709F090E0892FFB
:1007B0000895CF92DF92EF92FF92CF930E94CF03E2
:1007C000882309F463C084ED9FE00E94E10090E07B
:1007D00090936B3880936A3885ED9FE00E94E1002A
:1007E00090E090931D0180931C0186ED9FE00E9494
:1007F000E10090E090931B0180931A018BED9FE044
:100800000E94E100C82F8CED9FE00E94E100C82EFD
:10081000D12CE12CF12C7601DD24CC24FC2A8DEDA9
:100820009FE00E94E100C82F8EED9FE00E94E10052
:10083000C82ADC2AC0926238D0926338E0926438C9
:10084000F092653887ED9FE00E94E100C82F88EDA7
:100850009FE00E94E100C82ED12CE12CF12C760102
:10086000DD24CC24FC2A89ED9FE00E94E100C82F02
:100870008AED9FE00E94E100C82ADC2AC092663817
:10088000D0926738E0926838F0926938CF91FF9043
:10089000EF90DF90CF90089580916038882309F41D
:1008A0008AC080916138882309F485C060916A38D4
:1008B00084ED9FE00E94CD0060911C0185ED9FE0DA
:1008C0000E94CD0060911A0186ED9FE00E94CD004C
:1008D0008091663890916738A0916838B0916938F6
:1008E0006B2F77278827992787ED9FE00E94CD00FF
:1008F0008091663890916738A0916838B0916938D6
:10090000BD018827992788ED9FE00E94CD00809146
:10091000663890916738A0916838B0916938692F2E
:100920007A2F8B2F992789ED9FE00E94CD0060914F
:1009300066388AED9FE00E94CD00809162389091E8
:100940006338A0916438B09165386B2F772788277A
:1009500099278BED9FE00E94CD00809162389091A5
:100960006338A0916438B0916538BD018827992714
:100970008CED9FE00E94CD008091623890916338A9
:10098000A0916438B0916538692F7A2F8B2F992701
:100990008DED9FE00E94CD00609162388EED9FE06A
:1009A0000E94CD0063E78FED9FE00E94CD008AE0BA
:1009B00090E00C9466018AE090E00C94350160E0D0
:1009C0008FED9FE00C94CD0082E390E00E94FA004E
:1009D0000E9449038CE698E30E94CA201092613875
:1009E00008958091623890916338A0916438B091F5
:1009F0006538892B8A2B8B2BE1F08091663890919A
:100A00006738A0916838B0916938892B8A2B8B2B75
:100A100081F080911A0190911B018F3F910549F05F
:100A200080916A3890916B38892B19F010921901D6
:100A3000089581E080931901089581E040916B0150
:100A400050916C012091690130916A01421753075E
:100A500009F480E0089580916B0190916C010196FA
:100A600069E170E00E94882AAC0181E0209169016F
:100A700030916A014217530709F080E00895CF933F
:100A80008CE698E30E942E1FC82F0E94782760935F
:100A90005D0170935E0180935F0190936001C0FFE0
:100AA00008C081E0809368018093670180936601AC
:100AB00006C01092680110926701109266012091A1
:100AC00068018091610190916201211108C020911B
:100AD0006701211104C0209166012223B1F0209109
:100AE0001301309114018217930748F401969093F3
:100AF00062018093610181E08093650112C081E011
:100B000080936501809364010CC0009731F00197D8
:100B1000909362018093610102C01092640110926F
:100B2000650180916401882319F0CF910C94EA004B
:100B3000CF910C94EE000F931F930E9478270091A1
:100B40005D0110915E0120915F0130916001DC0137
:100B5000CB01801B910BA20BB30B00910F011091E5
:100B60001001209111013091120180179107A20705
:100B7000B30720F01F910F910C943F051F910F9127
:100B8000089580910901809353010895803C41F4B8
:100B90006BED70E08EE898E30E94E3008CED09C0F5
:100BA0008B3D39F46BED70E08EE898E30E94E30032
:100BB0008DED682F8EE898E30C94702460EC70E063
:100BC0008EE898E30E94E30061E270E08EE898E32B
:100BD0000E94E300809174010E94C6058091730118
:100BE0000E94C605809172010E94C6058091710124
:100BF0000E94C60560EC70E08EE898E30C94E30078
:100C000060EC70E08EE898E30E94E30062E270E03E
:100C10008EE898E30E94E300809170010E94C6056F
:100C200080916F010E94C60580916E010E94C605E9
:100C300080916D010E94C60560EC70E08EE898E33B
:100C40000C94E30060EC70E08EE898E30E94E3000F
:100C500062E070E08EE898E30E94E30080916938DA
:100C60000E94C605809168380E94C6058091673849
:100C70000E94C605809166380E94C60560EC70E04F
:100C80008EE898E30C94E30060EC70E08EE898E363
:100C90000E94E30061E070E08EE898E30E94E300C8
:100CA000809165380E94C605809164380E94C6050F
:100CB000809163380E94C605809162380E94C60503
:100CC00060EC70E08EE898E30C94E300CF93DF9340
:100CD000C8E3DFE0CE010E94E1000E94C605219634
:100CE000C11580E1D807B1F7DF91CF91089560EC8D
:100CF00070E08EE898E30E94E30061E570E08EE822
:100D000098E30E94E3000E94660660EC70E08EE8C3
:100D100098E30C94E300CF93C82F60EC70E08EE86A
:100D200098E30E94E30060E970E08EE898E30E9497
:100D3000E3006C2F8EE898E30E94702460EC70E072
:100D40008EE898E3CF910C94E300CF93DF93C82F04
:100D5000D62F0E945903811102C0C83C28F083E0BD
:100D6000DF91CF910C948B068C2F90E06D2F885CD7
:100D7000904FDF91CF910C94CD000E94F1048091AF
:100D80006138811144C08091190181113CC080916A
:100D900060388823C1F14091623850916338609186
:100DA0006438709165388CE698E30E948A22892B1A
:100DB00041F481E00E948B0680E090E00E94FA00FE
:100DC000089581E0809361380E94D6020E94080352
:100DD0000E94BC020E94C9020E941B038CE698E399
:100DE0000E941C2264E17AE08CE698E30E945E2077
:100DF00060E070E08CE698E30E946E2283E090E071
:100E00000E946601089583E090E00E9435010895F4
:100E10000E945903882361F00E946303882341F0F4
:100E20000E946D03882321F00E947C03811103C07E
:100E30001092603808950E948903882371F081E040
:100E4000809360380E94CF03882339F00E94D90331
:100E500082E1809318010C94BD06089580E00E9401
:100E60008F290E94EB2526E040E052EC61E070E023
:100E70008EE898E30E94D92461E08CE00E945C280F
:100E800061E08DE00E945C2884EF91E0E7E6F6E304
:100E9000DF019C011D9221503040E1F7E3E7F4E3CC
:100EA000DF019C011D9221503040E1F784E0EFE624
:100EB000F4E3DF011D928A95E9F784ED90E3E7EA18
:100EC000F1E0DF019C011D9221503040E1F782E307
:100ED000E5E7F1E0DF011D928A95E9F722E030E0D5
:100EE00043E050E064E070E08CE698E30E94D61E98
:100EF0000C940807CF93DF93EC0120916B013091A4
:100F00006C01C901019669E170E00E94882A409154
:100F1000690150916A018417950749F1F901EE0FB3
:100F2000FF1FEB58FE4FD183C08344EF51E0249F55
:100F3000F001259FF00D349FF00D1124E955FE4F6F
:100F4000A3E7B4E39D01235734432C173D0718F45E
:100F50002D912193F7CF90936C0180936B010E94A8
:100F60002B05811109C0DF91CF910C944F0284E0D1
:100F7000DF91CF910C948B06DF91CF910895CF93A1
:100F8000C0911601CC5D60EC70E08EE898E30E94A1
:100F9000E30063E270E08EE898E30E94E3006C2FC8
:100FA0008EE898E30E94702460EC70E08EE898E38D
:100FB000CF910C94E30060EC70E08EE898E30E941F
:100FC000E30064E070E08EE898E30E94E300609143
:100FD0006A388EE898E30E94702460EC70E08EE836
:100FE00098E30C94E30060EC70E08EE898E30E94D4
:100FF000E30065E070E08EE898E30E94E300609112
:101000001C018EE898E30E94702460EC70E08EE88A
:1010100098E30C94E30060EC70E08EE898E30E94A3
:10102000E30063E070E08EE898E30E94E3006091E3
:101030001A018EE898E30E94702460EC70E08EE85C
:1010400098E30C94E300CF93C82F60EC70E08EE837
:1010500098E30E94E30060E470E08EE898E30E9469
:10106000E3006C2F8EE898E30E94702460EC70E03F
:101070008EE898E3CF910C94E30090915A01992364
:1010800071F0803CD1F480910E0181110BC010925F
:101090005A0180915B0190915C010C947A07803C2D
:1010A00009F0A0C181E080935A018EEF80930E0178
:1010B00010925C0110925B01089520915B013091C8
:1010C0005C01243F91E0390708F08CC190910E013A
:1010D0002115310529F49E3F19F480930E010895DE
:1010E00091111FC08B3D21F481E080935901089537
:1010F00090915901992349F08C3D21F08D3D19F4CF
:101100008BED01C080EC10925901A9014F5F5F4F38
:1011100050935C0140935B01F901ED58FB4C8083D7
:101120000895913009F044C08B3D19F49093590112
:1011300018C090915901992349F08C3D21F08D3DC3
:1011400019F48BED01C080EC10925901A9014F5F99
:101150005F4F50935C0140935B01F901E159FB4CF7
:10116000808380915B0190915C01049709F03AC102
:1011700060916F34709170348091713490917234B9
:101180000E94E62A611571058105910511F40C9400
:101190004406609362387093633880936438909308
:1011A000653880911801813191F70E942C03EFCFAF
:1011B000923009F045C08B3D21F481E080935901C4
:1011C00018C090915901992349F08C3D21F08D3D33
:1011D00019F48BED01C080EC10925901A9014F5F09
:1011E0005F4F50935C0140935B01F901E159FB4C67
:1011F000808380915B0190915C01049709F0F2C0BB
:1012000060916F3470917034809171349091723428
:101210000E94E62A611571058105910511F40C946F
:10122000220660936638709367388093683890938D
:10123000693880911801813191F70E940803EFCF3E
:101240009330A9F48F3F11F40C940B08823110F401
:1012500090E002C081E190E090931B0180931A011D
:1012600080911801813181F70E94D602EDCF943030
:10127000D1F48F3F11F40C94DB07863038F0282F1F
:1012800030E08D3028F02CE030E002C026E030E085
:1012900030936B3820936A3880911801813159F767
:1012A0000E94BC02E8CF9530D1F48F3F11F40C942A
:1012B000F307853038F0282F30E0893028F028E017
:1012C00030E002C025E030E030931D0120931C0186
:1012D00080911801813159F70E94C902E8CF9630F8
:1012E00071F48F3F21F0811104C00E94EA040C9434
:1012F0001D02813009F076C00E94BD06F8CF913200
:1013000011F40C94DE05923211F40C940006933221
:1013100011F40C94BF07973021F40E94F1040C944F
:101320003602903319F490E00C946601903421F465
:101330000E943F030C942308983029F4833709F066
:1013400051C00C9486029E3059F4813019F4809378
:101350005F3804C0811102C010925F380C9467029C
:10136000993521F4883FF1F50E94E404913511F498
:101370000C947706923551F58B3D21F481E08093F2
:10138000590118C090915901992349F08C3D21F0E1
:101390008D3D19F48BED01C080EC10925901A9012B
:1013A0004F5F5F4F50935C0140935B01F901E1593E
:1013B000FB4C808380915B0190915C01029791F4DA
:1013C0006091703480916F340C94A506903511F4BF
:1013D0000C949E02933511F40C944C04943511F442
:1013E0000C94DF0408950F931F93CF93DF938C0128
:1013F00001151105A1F0C0915B38D0915C38CE0188
:10140000019690935C3880935B388CE698E30E9459
:10141000601FC959D94C888301501109E9CFDF9168
:10142000CF911F910F910895CF93DF93EC0180919D
:101430005F3881112BC08CE698E30E94601F2197D2
:101440004091150180FF0DC09C01332754E0359574
:1014500027955A95E1F74F3F09F497C0241395C09B
:101460007BC04F3F39F010925C3810925B388FEFA1
:10147000809315018CE698E30E94311F9093170129
:1014800080931601CE010E94F30992C010925C383D
:1014900010925B388CE698E30E94311F90931701FD
:1014A00080931601CE010E94F30960EC70E08EE893
:1014B00098E30E94E30063E270E08EE898E30E9404
:1014C000E3006091160164528EE898E30E94702454
:1014D00060EC70E08EE898E30E94E30060EC70E05E
:1014E0008EE898E30E94E30060E070E08EE898E305
:1014F0000E94E300C7E6D6E320915B3830915C3868
:10150000CE01875696438217930768F060EC70E02F
:101510008EE898E30E94E30010925C3810925B38EA
:10152000DF91CF9108956991603C41F46BED70E0DB
:101530008EE898E30E94E3006CED09C06B3D39F43E
:101540006BED70E08EE898E30E94E3006DED8EE8AD
:1015500098E30E947024D0CF8CE698E30E94311F5C
:101560002091160130911701820F931F97FD01966C
:10157000959587959093170180931601CE010E944F
:10158000F3098FEF8093150113C010925C3810920D
:101590005B38209315018CE698E30E94311F9093ED
:1015A000170180931601CE01DF91CF910C94F309BE
:1015B00060EC70E08EE898E30E94E30063E270E084
:1015C0008EE898E30E94E3006091160164528EE871
:1015D00098E30E94702460EC70E08EE898E30E942B
:1015E000E30060EC70E08EE898E30E94E30060E0C6
:1015F00070E08EE898E30E94E300C7E6D6E320910E
:101600005B3830915C38CE0187569643821793073A
:1016100008F07CCF6991603C41F46BED70E08EE89E
:1016200098E30E94E3006CED09C06B3D39F46BED6B
:1016300070E08EE898E30E94E3006DED8EE898E399
:101640000E947024DCCFCF92DF92EF92FF920F9333
:101650001F93CF93DF93EC0180916138882309F4C5
:101660007AC080915F38811158C00E94F20060E01A
:1016700071E080E090E00E94F325162F107FCF3FAD
:10168000D10508F0116060E070E08CE698E30E94FC
:101690004D22612F8CE698E30E94901E9BE7C92E95
:1016A00092E3D92EEE24E394F12CC6018B5792439A
:1016B0008C179D07F0F4F60161916F018CE698E3B9
:1016C0000E94901EFFEFEF1AFF0A8FEFE816F10459
:1016D00061F78CE698E30E94E31F60E070E08CE61F
:1016E00098E30E944D22612F8CE698E30E94901EA1
:1016F000D9CF8CE698E30E94E31F0E94F60060E0D9
:1017000070E08CE698E3DF91CF911F910F91FF90ED
:10171000EF90DF90CF900C946E220E94F200CF3FAA
:10172000D10519F010F0CFEFD0E060E070E08CE66A
:1017300098E30E944D220BE712E3C8018B579243B6
:101740008C179D07B0F6F80161918F018CE698E344
:101750000E94901EF2CF82E00E948B0685E090E00E
:10176000DF91CF911F910F91FF90EF90DF90CF907D
:101770000C94FA00CF93DF938091690190916A01F4
:1017800024EF31E0829FF001839FF00D929FF00DD6
:1017900011249C01220F331FD901AB58BE4FCD91AC
:1017A000DC91ABE7B2E3E955FE4FBF01AF01461B49
:1017B000570B4C175D0720F440814D931192F6CFE3
:1017C000F901EB58FE4F11821082019669E170E039
:1017D0000E94882A90936A0180936901CE010E9439
:1017E000230B0E942B05811104C0DF91CF910C9433
:1017F0004F02DF91CF9108950F931F93809161382D
:10180000882359F00E949B050E941D05882381F0C2
:101810008091580181110CC04AC0809160388823A2
:1018200019F00E94930104C00E94D8010E94EA04AA
:101830008EE898E30E940224892BA1F081E0809336
:1018400058018EE898E30E941C240E943D080E94E3
:1018500078276093540170935501809356019093BB
:1018600057014CC080915801882309F447C00E9459
:101870007827009154011091550120915601309123
:101880005701DC01CB01801B910BA20BB30B009124
:101890000A0110910B0120910C0130910D0180176C
:1018A0009107A207B30750F11092580127C0809109
:1018B0006301811102C00E943F0580916501811181
:1018C00019C080916401811115C080916301882342
:1018D00031F062E370E080E090E00E94A9270E946E
:1018E0003F05809165018111A3CF109263010E9491
:1018F000BA0B9ECF81E0809363019ACF1F910F9125
:1019000008952F923F924F925F926F927F928F92A3
:101910009F92AF92BF92CF92DF92EF92FF920F937E
:101920001F93CF93DF93CDB7DEB7C457D1090FB65E
:10193000F894DEBF0FBECDBFE5969FAF8EAFE597A3
:10194000E3967FAF6EAFE3971A01DC0118964D90D6
:101950005D906D907C901B9761964CAE5DAE6EAEC7
:101960007FAE61971C964D905D906D907C901F9717
:1019700049825A826B827C8250964D905D906D9028
:101980007C9053974D825E826F82788654964D90FC
:101990005D906D907C90579749865A866B867C86C1
:1019A000A85ABF4F6396BFAFAEAF6397FC01E45A2E
:1019B000FF4F6596FFAFEEAF6597805A9F4F6796D2
:1019C0009FAF8EAF6797E596AEADBFADE597AC59CB
:1019D000BF4F6996BFAFAEAF6997E596EEADFFAD6D
:1019E000E597E859FF4F6B96FFAFEEAF6B97E59623
:1019F0008EAD9FADE59784599F4F6D969FAF8EAF8B
:101A00006D97E596AEADBFADE597A059BF4F6F9608
:101A1000BFAFAEAF6F97E596EEADFFADE597EC5873
:101A2000FF4FA196FFAFEEAFA197E5968EAD9FADAC
:101A3000E59788589F4FA3969FAF8EAFA397E596E3
:101A4000AEADBFADE597A458BF4FA596BFAFAEAF43
:101A5000A597E596EEADFFADE597E058FF4FA79649
:101A6000FFAFEEAFA797E5968EAD9FADE5978C578C
:101A70009F4FA9969FAF8EAFA997E596AEADBFAD2C
:101A8000E597A857BF4FAB96BFAFAEAFAB97E59604
:101A9000EEADFFADE597E457FF4FAD96FFAFEEAF6C
:101AA000AD97E5968EAD9FADE59780579F4FAF966A
:101AB0009FAF8EAFAF97E596AEADBFADE597AC5695
:101AC000BF4FE196BFAFAEAFE197E396AEADBFAD0E
:101AD000E3974D905D906D907C904D865E866F860D
:101AE000788A6396EEADFFAD639740825182628241
:101AF00073820D811E812F81388549845A846B84BD
:101B00007C84042515252625372569807A808B80DD
:101B10009C80062117212821392189849A84AB844D
:101B2000BC84082519252A253B2561968CAD9DADE1
:101B3000AEADBFAD619788589B45A549B8424D856C
:101B40005E856F857889840F951FA61FB71F080FC4
:101B5000191F2A1F3B1FD901C80147E0880F991F91
:101B6000AA1FBB1F4A95D1F759E1369527951795BE
:101B700007955A95D1F7082B192B2A2B3B2B6981F6
:101B80007A818B819C81060F171F281F391FE396CE
:101B9000AEADBFADE39714968D919D910D90BC9124
:101BA000A02D898B9A8BAB8BBC8B6596EEADFFAD70
:101BB000659780839183A283B383C980DA80EB80A9
:101BC000FC804D805E806F807884C424D524E62418
:101BD000F724C022D122E222F322C424D524E62411
:101BE000F724D501C4018A5A9844A843B7416988AB
:101BF0007A888B889C88860D971DA81DB91DC80EF4
:101C0000D91EEA1EFB1ED701C6016CE0880F991F82
:101C1000AA1FBB1F6A95D1F774E1F694E794D79495
:101C2000C7947A95D1F7C82AD92AEA2AFB2AC00E86
:101C3000D11EE21EF31EE396AEADBFADE39718963C
:101C40008D909D90AD90BC901B978D8A9E8AAF8A97
:101C5000B88E6796EEADFFAD679780829182A282C3
:101C6000B38249815A816B817C8140275127622749
:101C700073274C215D216E217F2149805A806B8022
:101C80007C8044255525662577258D819E81AF81F1
:101C9000B88585529F48AF4DBB4D880D991DAA1D33
:101CA000BB1D480F591F6A1F7B1FDB01CA01EFE0F4
:101CB000B695A79597958795EA95D1F7F1E1440FE9
:101CC000551F661F771FFA95D1F7482B592B6A2BA2
:101CD0007B2B4C0D5D1D6E1D7F1DE396AEADBFAD24
:101CE000E3971C966D907D908D909C901F97698EC8
:101CF0007A8E8B8E9C8E6996EEADFFAD6997608271
:101D0000718282829382480159018C249D24AE24E1
:101D1000BF2484229522A622B72280269126A226BD
:101D2000B32689819A81AB81BC8182519143A244BF
:101D3000BE43498C5A8C6B8C7C8C840D951DA61DE2
:101D4000B71D880E991EAA1EBB1ED501C401EAE06C
:101D5000B695A79597958795EA95D1F7F6E1880C02
:101D6000991CAA1CBB1CFA95D1F7882A992AAA2A81
:101D7000BB2A840E951EA61EB71EE396AEADBFAD60
:101D8000E39750968D919D910D90BC91A02D8D8FD4
:101D90009E8FAF8FB8A36B96EEADFFAD6B97808330
:101DA0009183A283B3838155904FA348BA40080F13
:101DB000191F2A1F3B1FD701C60184279527A62775
:101DC000B72788219921AA21BB218C259D25AE25E5
:101DD000BF25080F191F2A1F3B1FD901C801E7E0C3
:101DE000880F991FAA1FBB1FEA95D1F7F9E1369515
:101DF000279517950795FA95D1F7082B192B2A2BBC
:101E00003B2B080D191D2A1D3B1DE396AEADBFAD42
:101E1000E39754964D905D906D907C90579749A2B2
:101E20005AA26BA27CA26D96EEADFFAD6D9740827B
:101E3000518262827382D301C201865D9943A847B1
:101E4000B84BC80ED91EEA1EFB1EDB01CA0188254D
:101E50009925AA25BB2580239123A223B323842778
:101E60009527A627B727C80ED91EEA1EFB1ED70145
:101E7000C601ECE0880F991FAA1FBB1FEA95D1F796
:101E8000F4E1F694E794D794C794FA95D1F7C82A69
:101E9000D92AEA2AFB2AC00ED11EE21EF31EE396BF
:101EA000AEADBFADE39758964D905D906D907C9030
:101EB0005B974DA25EA26FA278A66F96EEADFFADC6
:101EC0006F974082518262827382D301C2018D5E1C
:101ED000994BAF4CB745480F591F6A1F7B1FD5015F
:101EE000C40180279127A227B3278C219D21AE21F1
:101EF000BF2188259925AA25BB25480F591F6A1F90
:101F00007B1FDB01CA01EFE0B695A79597958795F2
:101F1000EA95D1F7F1E1440F551F661F771FFA9537
:101F2000D1F7482B592B6A2B7B2B4C0D5D1D6E1D59
:101F30007F1DE396AEADBFADE3975C964D905D908F
:101F40006D907C905F9749A65AA66BA67CA6A19639
:101F5000EEADFFADA1974082518262827382D301C0
:101F6000C2018F5F9A46A94BB240880E991EAA1EE5
:101F7000BB1ED901C8018C259D25AE25BF25842314
:101F80009523A623B72380279127A227B327880E5E
:101F9000991EAA1EBB1ED501C401EAE0B695A795FD
:101FA00097958795EA95D1F7F6E1880C991CAA1CBC
:101FB000BB1CFA95D1F7882A992AAA2ABB2A840E33
:101FC000951EA61EB71EE396AEADBFADE3979096E5
:101FD0004D905D906D907C9093974DA65EA66FA6F8
:101FE00078AAA396EEADFFADA3974082518262829C
:101FF0007382D301C20188529746AF47B649080F92
:10200000191F2A1F3B1FD701C60184279527A62722
:10201000B72788219921AA21BB218C259D25AE2592
:10202000BF25080F191F2A1F3B1FD901C801E7E070
:10203000880F991FAA1FBB1FEA95D1F7F9E13695C2
:10204000279517950795FA95D1F7082B192B2A2B69
:102050003B2B080D191D2A1D3B1DE396AEADBFADF0
:10206000E39794964D905D906D907C90979749AAD8
:102070005AAA6BAA7CAAA596EEADFFADA5974082A1
:10208000518262827382D301C20181559840AB4B69
:10209000B447C80ED91EEA1EFB1EDB01CA01882503
:1020A0009925AA25BB2580239123A223B323842726
:1020B0009527A627B727C80ED91EEA1EFB1ED701F3
:1020C000C601ECE0880F991FAA1FBB1FEA95D1F744
:1020D000F4E1F694E794D794C794FA95D1F7C82A17
:1020E000D92AEA2AFB2AC00ED11EE21EF31EE3966D
:1020F000AEADBFADE39798964D905D906D907C909E
:102100009B974DAA5EAA6FAA78AEA796EEADFFADDB
:10211000A7974082518262827382D301C2018F5499
:10212000944AA109B109480F591F6A1F7B1FD501A5
:10213000C40180279127A227B3278C219D21AE219E
:10214000BF2188259925AA25BB25480F591F6A1F3D
:102150007B1FDB01CA01EFE0B695A79597958795A0
:10216000EA95D1F7F1E1440F551F661F771FFA95E5
:10217000D1F7482B592B6A2B7B2B4C0D5D1D6E1D07
:102180007F1DE396AEADBFADE3979C964D905D90FD
:102190006D907C909F9749AE5AAE6BAE7CAEA9967F
:1021A000EEADFFADA9974082518262827382D30166
:1021B000C20182549842A34AB647880E991EAA1EAD
:1021C000BB1ED901C8018C259D25AE25BF258423C2
:1021D0009523A623B72380279127A227B327880E0C
:1021E000991EAA1EBB1ED501C401EAE0B695A795AB
:1021F00097958795EA95D1F7F6E1880C991CAA1C6A
:10220000BB1CFA95D1F7882A992AAA2ABB2A840EE0
:10221000951EA61EB71EE396AEADBFADE397D09652
:102220004D905D906D907C90D39721964CAE5DAEB5
:102230006EAE7FAE2197AB96EEADFFADAB97408211
:10224000518262827382FEED4F1AFEEE5F0AFFE654
:102250006F0AF4E97F0A040D151D261D371D26019E
:1022600037014426552666267726482059206A20BD
:102270007B204C245D246E247F24040D151D261D17
:10228000371D2801390187E0440C551C661C771C5A
:102290008A95D1F799E136952795179507959A95DF
:1022A000D1F70429152926293729080D191D2A1DBA
:1022B0003B1DD4964D905D906D907C90D797259660
:1022C0004CAE5DAE6EAE7FAE2597AD96EEADFFAD7A
:1022D000AD974082518262827382FDE64F1AFEE81A
:1022E0005F0AF7E66F0AF2E07F0AC40CD51CE61C11
:1022F000F71C2A013B01482459246A247B244022EC
:102300005122622273224426552666267726C40C63
:10231000D51CE61CF71C26013701ECE0440C551CCB
:10232000661C771CEA95D1F7F4E1F694E794D7940C
:10233000C794FA95D1F7C428D528E628F728C00E07
:10234000D11EE21EF31ED8964D905D906D907C904C
:10235000DB9729964CAE5DAE6EAE7FAE2997AF96F9
:10236000EEADFFADAF974082518262827382F2E799
:102370004F1AFCEB5F0AF6E86F0AF9E57F0A440D95
:10238000551D661D771D2401350140265126622604
:1023900073264C205D206E207F20482459246A2417
:1023A0007B24440D551D661D771D2A013B018FE0DE
:1023B00076946794579447948A95D1F791E1440FA6
:1023C000551F661F771F9A95D1F74429552966290D
:1023D00077294C0D5D1D6E1D7F1DDC964D905D9027
:1023E0006D907C90DF972D964CAE5DAE6EAE7FAE5D
:1023F0002D97E196EEADFFADE1974082518262826A
:102400007382FFED4F1AF7EF5F0AFBE46F0AF6EBFA
:102410007F0A840C951CA61CB71C280139014C248A
:102420005D246E247F244422552266227722402692
:10243000512662267326840C951CA61CB71C240109
:102440003501EAE07694679457944794EA95D1F77A
:10245000F6E1880C991CAA1CBB1CFA95D1F78428BC
:102460009528A628B728840E951EA61EB71E498853
:102470005A886B887C888EE9481A8AED580A81EE62
:10248000680A89E0780A040D151D261D371D2A01EA
:102490003B01482459246A247B244C205D206E2073
:1024A0007F204426552666267726040D151D261DF9
:1024B000371D28013901A5E0440C551C661C771C0A
:1024C000AA95D1F7BBE13695279517950795BA954B
:1024D000D1F70429152926293729080D191D2A1D88
:1024E0003B1D4DA05EA06FA078A490EC491A9CE41F
:1024F000590A9FEB690A9FE3790AC40CD51CE61CB4
:10250000F71C2401350140265126622673264422F9
:10251000552266227722482459246A247B24C40C3D
:10252000D51CE61CF71C2601370189E0440C551C1C
:10253000661C771C8A95D1F797E1F694E794D794B7
:10254000C7949A95D1F7C428D528E628F728C00E55
:10255000D11EE21EF31E49AC5AAC6BAC7CACAFEAA8
:102560004A1AA5EA5A0AA1EA6A0AA9ED7A0A440DAA
:10257000551D661D771D280139014C245D246E24EC
:102580007F24482059206A207B204026512662263D
:102590007326440E551E661E771ED301C2014EE0FF
:1025A000880F991FAA1FBB1F4A95D1F752E1769455
:1025B0006794579447945A95D1F7482A592A6A2A1A
:1025C0007B2A4C0C5D1C6E1C7F1C4D855E856F85C7
:1025D00078894655584369447641840E951EA61E57
:1025E000B71EB701A601442555256625772540234A
:1025F0005123622373234C255D256E257F25480DCD
:10260000591D6A1D7B1DDB01CA01ECE0B695A7953B
:1026100097958795EA95D1F7F4E1440F551F661F0A
:10262000771FFA95D1F7482B592B6A2B7B2B440D3A
:10263000551D661D771D89A09AA0ABA0BCA0B3EA6A
:102640008B1ABFEE9B0AB0EDAB0AB9E2BB0A080DCC
:10265000191D2A1D3B1D5301420184269526A626DD
:10266000B7268C209D20AE20BF2084249524A6244C
:10267000B724080D191D2A1D3B1D48015901A5E06D
:10268000880C991CAA1CBB1CAA95D1F7BBE13695F6
:10269000279517950795BA95D1F7082919292A2959
:1026A0003B29040F151F261F371F8DA89EA8AFA812
:1026B000B8ACEDEA8E1AEBEE9E0AEBEBAE0AEDEF4C
:1026C000BE0AC80CD91CEA1CFB1C4A015B0180260F
:1026D0009126A226B32684209520A620B720842602
:1026E0009526A626B726C80CD91CEA1CFB1C460159
:1026F000570189E0880C991CAA1CBB1C8A95D1F74C
:1027000097E1F694E794D794C7949A95D1F7C8289F
:10271000D928EA28FB28C00ED11EE21EF31E2D96F2
:102720008CAC9DACAEACBFAC2D97FFE78F1AF9E136
:102730009F0AFEE5AF0AF7E2BF0A480C591C6A1C63
:102740007B1C480159018C249D24AE24BF24842283
:102750009522A622B72280269126A226B326480CCF
:10276000591C6A1C7B1C53014201EEE0880C991C29
:10277000AA1CBB1CEA95D1F7F2E1769467945794B2
:102780004794FA95D1F7482859286A287B284C0C99
:102790005D1C6E1C7F1C8D8C9E8CAF8CB8A088E35A
:1027A000881A84E0980A8CE2A80A88E1B80A480DE1
:1027B000591D6A1D7B1D4601570184249524A624BA
:1027C000B72480229122A222B3228C249D24AE24FD
:1027D000BF24480D591D6A1D7B1D4A015B01ACE0F9
:1027E000B694A79497948794AA95D1F7B4E1440F2F
:1027F000551F661F771FBA95D1F7482959296A29AD
:102800007B29440D551D661D771D89A89AA8ABA884
:10281000BCA89AE1891A92E3990A9EE1A90A9EED61
:10282000B90A080D191D2A1D3B1D530142018426BA
:102830009526A626B7268C209D20AE20BF20842476
:102840009524A624B724080D191D2A1D3B1D4801F7
:10285000590185E0880C991CAA1CBB1C8A95D1F7EC
:102860009BE136952795179507959A95D1F70829F5
:1028700019292A293B29040F151F261F371F2996BE
:102880008CAC9DACAEACBFAC2997AAE28A1AA8EF7B
:102890009A0AA8ECAA0AACE3BA0AC80CD91CEA1C2A
:1028A000FB1C4A015B0180269126A226B3268420C8
:1028B0009520A620B72084269526A626B726C80CE4
:1028C000D91CEA1CFB1C46015701E9E0880C991C45
:1028D000AA1CBB1CEA95D1F7F7E1F694E794D794CC
:1028E000C794FA95D1F7C828D928EA28FB28C00E42
:1028F000D11EE21EF31E898C9A8CAB8CBC8CB9E77E
:102900008B1AB2EF9B0ABAE2AB0ABBE0BB0A480CD7
:10291000591C6A1C7B1C480159018C249D24AE243F
:10292000BF2484229522A622B72280269126A226A1
:10293000B326480C591C6A1C7B1C53014201AEE0B3
:10294000880C991CAA1CBB1CAA95D1F7B2E17694FD
:10295000679457944794BA95D1F7482859286A281C
:102960007B284C0C5D1C6E1C7F1C8DA49EA4AFA408
:10297000B8A8E3E18E1AEBEE9E0AE5EAAE0AEAEBAE
:10298000BE0A480D591D6A1D7B1D4601570184244E
:102990009524A624B72480229122A222B3228C243B
:1029A0009D24AE24BF24480D591D6A1D7B1D4A017C
:1029B0005B018CE0B694A794979487948A95D1F79D
:1029C00094E1440F551F661F771F9A95D1F7482948
:1029D00059296A297B29440D551D661D771D2596A9
:1029E0008CAC9DACAEACBFAC2597FBEF8F1AF6E17B
:1029F0009F0AFCE1AF0AF6E5BF0A080D191D2A1D62
:102A00003B1D5301420184269526A626B7268C201D
:102A10009D20AE20BF2084249524A624B724080D31
:102A2000191D2A1D3B1D48015901E5E0880C991C20
:102A3000AA1CBB1CEA95D1F7FBE1369527951795A3
:102A40000795FA95D1F7082919292A293B29040F56
:102A5000151F261F371F8D889E88AF88B88C88E089
:102A6000881A8CE5980A80E1A80A83E0B80AC80CA5
:102A7000D91CEA1CFB1C4A015B0180269126A22678
:102A8000B32684209520A620B72084269526A62646
:102A9000B726C80CD91CEA1CFB1C46015701A9E04B
:102AA000880C991CAA1CBB1CAA95D1F7B7E1F69417
:102AB000E794D794C794BA95D1F7C828D928EA28BB
:102AC000FB28C00ED11EE21EF31E89A49AA4ABA45B
:102AD000BCA497E2891A9DEF990A90E9A90A98E99E
:102AE000B90A480C591C6A1C7B1C480159018C24EA
:102AF0009D24AE24BF2484229522A622B7228026BC
:102B00009126A226B326480C591C6A1C7B1C530133
:102B100042018EE0880C991CAA1CBB1C8A95D1F737
:102B200092E176946794579447949A95D1F7482800
:102B300059286A287B284C0C5D1C6E1C7F1C4601A2
:102B4000570184249524A624B72421968CAD9DADED
:102B5000AEADBFAD21978657934BA54DB247480FF9
:102B6000591F6A1F7B1FD901C80188219921AA21F9
:102B7000BB218C259D25AE25BF25480F591F6A1FF7
:102B80007B1FDB01CA01ECE0B695A7959795879569
:102B9000EA95D1F7F4E1440F551F661F771FFA95A8
:102BA000D1F7482B592B6A2B7B2B440D551D661DE5
:102BB000771D89A19AA1ABA1BCA18E5B964CA540C3
:102BC000B109080F191F2A1F3B1F84269526A62628
:102BD000B726080D191D2A1D3B1D48015901A4E007
:102BE000880C991CAA1CBB1CAA95D1F7BCE1369590
:102BF000279517950795BA95D1F7082919292A29F4
:102C00003B29040F151F261F371F8DA49EA4AFA4B8
:102C1000B8A8AFE78A1AA9E09A0AAEE8AA0AA8E714
:102C2000BA0AC80CD91CEA1CFB1C530142018426B9
:102C30009526A626B72680269126A226B326C80C5E
:102C4000D91CEA1CFB1C460157018BE0880C991C1F
:102C5000AA1CBB1C8A95D1F795E1F694E794D7940A
:102C6000C7949A95D1F7C828D928EA28FB28C00E1E
:102C7000D11EE21EF31E89AC9AACABACBCACBEED6F
:102C80008B1ABEE99B0AB2E6AB0AB2E9BB0A480C52
:102C9000591C6A1C7B1C4A015B0180269126A226D6
:102CA000B3268C249D24AE24BF24480C591C6A1CD6
:102CB0007B1CF20123013F014C0C5D1C6E1C7F1C30
:102CC00029968CAC9DACAEACBFAC2997F4EF8F1AB3
:102CD000F7EC9F0AFAE1AF0AF2E0BF0A480D591D6E
:102CE0006A1D7B1D480159018C249D24AE24BF24FC
:102CF00084249524A624B724480D591D6A1D7B1DE4
:102D00004A015B01E9E0B694A79497948794EA9509
:102D1000D1F7F7E1440F551F661F771FFA95D1F7DA
:102D2000482959296A297B29440D551D661D771D9F
:102D300089889A88AB88BC888CEB881A85E1980AC8
:102D400081E4A80A8BE5B80A080D191D2A1D3B1D50
:102D50004601570184249524A624B7248426952669
:102D6000A626B726080D191D2A1D3B1D480159012D
:102D7000A4E0880C991CAA1CBB1CAA95D1F7BCE145
:102D80003695279517950795BA95D1F708291929EA
:102D90002A293B29040F151F261F371F8D8C9E8C57
:102DA000AF8CB8A097E5891A90E3990A91E2A90A35
:102DB00094EBB90AC80CD91CEA1CFB1C5301420154
:102DC00084269526A626B72680269126A226B326F7
:102DD000C80CD91CEA1CFB1C460157018BE0880C6F
:102DE000991CAA1CBB1C8A95D1F795E1F694E7942F
:102DF000D794C7949A95D1F7C828D928EA28FB28F0
:102E0000C00ED11EE21EF31E89A49AA4ABA4BCA4DA
:102E1000A0EA8A1AA4EB9A0AA4E4AA0AA9E0BA0AC8
:102E2000480C591C6A1C7B1C4A015B0180269126B8
:102E3000A226B3268C249D24AE24BF24480C591C02
:102E40006A1C7B1CF20123013F014C0C5D1C6E1CB3
:102E50007F1C8DA89EA8AFA8B8ACF0E98F1AF3E448
:102E60009F0AF0E4AF0AF1E4BF0A480D591D6A1D3C
:102E70007B1D480159018C249D24AE24BF24842449
:102E80009524A624B724840E951EA61EB71ED50130
:102E9000C40149E0B695A795979587954A95D1F7CE
:102EA00057E1880C991CAA1CBB1C5A95D1F7882A9B
:102EB000992AAA2ABB2A840C951CA61CB71C259605
:102EC0004CAD5DAD6EAD7FAD25974A53514864461C
:102ED000774D040F151F261F371FB701A601442584
:102EE000552566257725482559256A257B25040F14
:102EF000151F261F371FB901A801E4E0440F551F15
:102F0000661F771FEA95D1F7FCE13695279517954F
:102F10000795FA95D1F7042B152B262B372B080D87
:102F2000191D2A1D3B1D4D855E856F85788946508C
:102F3000584D6E457541C40ED51EE61EF71EB301F1
:102F4000A201482559256A257B254027512762275C
:102F500073274C0D5D1D6E1D7F1DDB01CA01EBE06B
:102F6000880F991FAA1FBB1FEA95D1F7F5E1769547
:102F7000679557954795FA95D1F7482B592B6A2BAA
:102F80007B2B400F511F621F731FC98CDA8CEB8C97
:102F9000FC8C8BE7C81A8FECD80A80E1E80A8BE238
:102FA000F80A4C0C5D1C6E1C7F1C75016401C02668
:102FB000D126E226F326C426D526E626F7264C0C93
:102FC0005D1C6E1C7F1CD20123013D01440E551E69
:102FD000661E771ECDA0DEA0EFA0F8A4BBEFCB1A33
:102FE000B2EEDB0AB7E7EB0ABBEFFB0A8C0C9D1CC9
:102FF000AE1CBF1C68017901C426D526E626F7263B
:10300000C424D524E624F7248C0C9D1CAE1CBF1CC4
:1030100075016401A9E0F694E794D794C794AA9542
:10302000D1F7B7E1880C991CAA1CBB1CBA95D1F743
:103030008C289D28AE28BF28840C951CA61CB71C84
:10304000C9A8DAA8EBA8FCA8E7ECCE1AEFE2DE0AE2
:10305000EBE2EE0AE6E2FE0A0C0D1D1D2E1D3F1DE1
:103060006A017B01C424D524E624F724C824D9248A
:10307000EA24FB240C0D1D1D2E1D3F1D6801790146
:1030800084E0CC0CDD1CEE1CFF1C8A95D1F79CE182
:1030900036952795179507959A95D1F70C291D29EF
:1030A0002E293F29080D191D2A1D3B1D2196CCAC48
:1030B000DDACEEACFFAC2197FBE1CF1AF6E6DF0A00
:1030C000F4E2EF0AF9E1FF0A4C0D5D1D6E1D7F1D54
:1030D00073016201C824D924EA24FB24C026D12626
:1030E000E226F3264C0D5D1D6E1D7F1D6A017B01DE
:1030F000EBE0CC0CDD1CEE1CFF1CEA95D1F7F5E1F2
:103100007695679557954795FA95D1F74C295D299E
:103110006E297F29400F511F621F731F2D96CCAC63
:10312000DDACEEACFFAC2D9788E0C81A83E8D80A76
:103130008DE5E80A80EEF80A4C0C5D1C6E1C7F1CC5
:1031400075016401C026D126E226F326C426D526C1
:10315000E626F7264C0C5D1C6E1C7F1CD201230159
:103160003D01440E551E661E771ECD88DE88EF8811
:10317000F88CBBE9CB1AB9EADB0AB3E5EB0ABBE38F
:10318000FB0A8C0C9D1CAE1CBF1C68017901C42677
:10319000D526E626F726C424D524E624F7248C0C6D
:1031A0009D1CAE1CBF1C75016401A9E0F694E79458
:1031B000D794C794AA95D1F7B7E1880C991CAA1C9B
:1031C000BB1CBA95D1F78C289D28AE28BF28840C4B
:1031D000951CA61CB71CCD84DE84EF84F888ECEB2C
:1031E000CE1AEDEDDE0AE6EDEE0AEBE0FE0A0C0D7E
:1031F0001D1D2E1D3F1D6A017B01C094D094E094DB
:10320000F094C828D928EA28FB28C424D524E62429
:10321000F7240C0D1D1D2E1D3F1D6801790186E050
:10322000CC0CDD1CEE1CFF1C8A95D1F79AE136957B
:103230002795179507959A95D1F70C291D292E29C1
:103240003F29080D191D2A1D3B1DC9A4DAA4EBA4B2
:10325000FCA4F9E6CF1AD108F5EDEF0AFCEBFF0A62
:103260004C0D5D1D6E1D7F1D73016201C094D094D5
:10327000E094F094C02AD12AE22AF32AC824D9245F
:10328000EA24FB244C0D5D1D6E1D7F1D6A017B0130
:10329000EAE0CC0CDD1CEE1CFF1CEA95D1F7F6E150
:1032A0007695679557954795FA95D1F74C295D29FD
:1032B0006E297F29400F511F621F731F2996CCACC6
:1032C000DDACEEACFFAC299789E5C81A8CEDD80AC5
:1032D0008BE6E80A84E5F80A4C0C5D1C6E1C7F1C2A
:1032E00075016401C094D094E094F094C42AD52A66
:1032F000E62AF72AC026D126E226F3264C0C5D1CCE
:103300006E1C7F1C73016201AFE0CC0CDD1CEE1C57
:10331000FF1CAA95D1F7B1E176946794579447942E
:10332000BA95D1F74C285D286E287F28440E551E8B
:10333000661E771EC9A0DAA0EBA0FCA097ECC91A04
:103340009FE5D90A9CE6E90A93E0F90A8C0C9D1CDA
:10335000AE1CBF1C68017901C094D094E094F09435
:10336000C428D528E628F728C426D526E626F72639
:103370008C0C9D1CAE1CBF1C750164018BE0F69487
:10338000E794D794C7948A95D1F795E1880C991C56
:10339000AA1CBB1C9A95D1F78C289D28AE28BF2863
:1033A000840C951CA61CB71C2196CCACDDACEEACF5
:1033B000FFAC2197ADE3CA1AA6EADA0AA4EAEA0A40
:1033C000AAE9FA0A0C0D1D1D2E1D3F1D6A017B0185
:1033D000C094D094E094F094C828D928EA28FB2817
:1033E000C424D524E624F7240C0D1D1D2E1D3F1DDD
:1033F00068017901E6E0CC0CDD1CEE1CFF1CEA95AF
:10340000D1F7FAE13695279517950795FA95D1F7F3
:103410000C291D292E293F29080D191D2A1D3B1D88
:10342000C98CDA8CEB8CFC8CBEE6CB1AB3E3DB0ADE
:10343000B3EFEB0AB0E7FB0A4C0D5D1D6E1D7F1D5F
:1034400073016201C094D094E094F094C02AD12A10
:10345000E22AF32AC824D924EA24FB244C0D5D1D5A
:103460006E1D7F1D6A017B01AAE0CC0CDD1CEE1CE9
:10347000FF1CAA95D1F7B6E17695679557954795C4
:10348000BA95D1F74C295D296E297F29400F511F2C
:10349000621F731FCDA8DEA8EFA8F8ACE3E8CE1A30
:1034A000EBE0DE0AE0E1EE0AF1084C0C5D1C6E1C5C
:1034B0007F1C75016401C094D094E094F094C42AF8
:1034C000D52AE62AF72AC026D126E226F3264C0C76
:1034D0005D1C6E1C7F1C730162018FE0CC0CDD1C37
:1034E000EE1CFF1C8A95D1F791E17694679457946E
:1034F00047949A95D1F74C285D286E287F28440E72
:10350000551E661E771EC988DA88EB88FC88FFE2A4
:10351000CF1AF2EADF0AFBE7EF0AFAE7FF0A8C0CA0
:103520009D1CAE1CBF1C68017901C094D094E0942E
:10353000F094C428D528E628F728C426D526E62600
:10354000F7268C0C9D1CAE1CBF1C75016401EBE0C2
:10355000F694E794D794C794EA95D1F7F5E1880CEF
:10356000991CAA1CBB1CFA95D1F78C289D28AE2863
:10357000BF28840C951CA61CB71CCDA4DEA4EFA408
:10358000F8A881EBC81A81E8D80A87E5E80A80E93B
:10359000F80A0C0D1D1D2E1D3F1D6A017B01C094F4
:1035A000D094E094F094C828D928EA28FB28C424B1
:1035B000D524E624F7240C0D1D1D2E1D3F1D68018A
:1035C0007901A6E0CC0CDD1CEE1CFF1CAA95D1F7FE
:1035D000BAE13695279517950795BA95D1F70C2935
:1035E0001D292E293F29080D191D2A1D3B1D2D9629
:1035F0008CAD9DADAEADBFAD2D9780529941A34D21
:10360000B140480F591F6A1F7B1FD301C20180952B
:103610009095A095B095802B912BA22BB32B88254C
:103620009925AA25BB25480F591F6A1F7B1FDB015F
:10363000CA01EAE0880F991FAA1FBB1FEA95D1F7BC
:10364000F6E17695679557954795FA95D1F7482B0A
:10365000592B6A2B7B2B400F511F621F731F8DA1AB
:103660009EA1AFA1B8A58C5E9C4BAE4FBC45480E49
:10367000591E6A1E7B1ED501C40180959095A095A8
:10368000B095842B952BA62BB72B80279127A227AB
:10369000B327480E591E6A1E7B1ED301C201EFE0FC
:1036A000880F991FAA1FBB1FEA95D1F7F1E1769405
:1036B000679457944794FA95D1F7482A592A6A2A69
:1036C0007B2A440E551E661E771E25968CAD9DAD39
:1036D000AEADBFAD25978F559E4EA74FB14B880E0F
:1036E000991EAA1EBB1ED901C80180959095A09570
:1036F000B09584299529A629B72984279527A62737
:10370000B727880E991EAA1EBB1ED501C401EBE087
:10371000B695A79597958795EA95D1F7F5E1880C29
:10372000991CAA1CBB1CFA95D1F7882A992AAA2AA7
:10373000BB2A840C951CA61CB71C8D8D9E8DAF8D4D
:10374000B8A18E579148AC4AB840080F191F2A1FDC
:103750003B1FDB01CA0180959095A095B095882903
:103760009929AA29BB2984259525A625B725080FBF
:10377000191F2A1F3B1FD901C801E6E0880F991FB6
:10378000AA1FBB1FEA95D1F7FAE136952795179541
:103790000795FA95D1F7082B192B2A2B3B2B080DEF
:1037A000191D2A1D3B1D89AD9AADABADBCAD8B5C1F
:1037B0009D40A54CB244480F591F6A1F7B1FD3017F
:1037C000C20180959095A095B095802B912BA22B4E
:1037D000B32B88259925AA25BB25480F591F6A1F99
:1037E0007B1FDB01CA01EAE0880F991FAA1FBB1FDC
:1037F000EA95D1F7F6E17695679557954795FA954D
:10380000D1F7482B592B6A2B7B2B400F511F621F7E
:10381000731F8D899E89AF89B88D85549D42A842BA
:10382000B54D480E591E6A1E7B1ED501C4018095F8
:103830009095A095B095842B952BA62BB72B802720
:103840009127A227B327480E591E6A1E7B1ED3015B
:10385000C201EFE0880F991FAA1FBB1FEA95D1F79D
:10386000F1E17694679457944794FA95D1F7482AF2
:10387000592A6A2A7B2A440E551E661E771E89A97C
:103880009AA9ABA9BCA98F569C42A947B441880EFE
:10389000991EAA1EBB1ED901C80180959095A095BE
:1038A000B09584299529A629B72984279527A62785
:1038B000B727880E991EAA1EBB1ED501C401EBE0D6
:1038C000B695A79597958795EA95D1F7F5E1880C78
:1038D000991CAA1CBB1CFA95D1F7882A992AAA2AF6
:1038E000BB2A61968CAD9DADAEADBFAD6197800F2B
:1038F000911FA21FB31F61968CAF9DAFAEAFBFAF3C
:103900006197840C951CA61CB71C89819A81AB8198
:10391000BC81880D991DAA1DBB1D89839A83AB8329
:10392000BC838D809E80AF80B884840C951CA61CBF
:10393000B71C8D829E82AF82B88689859A85AB85B9
:10394000BC85840F951FA61FB71F89879A87AB87F1
:10395000BC87E396AEADBFADE397A05CBF4FE396E7
:10396000BFAFAEAFE397B0E42B1A310811F00C945F
:10397000650D61964CAC5DAC6EAC7FAC6197E59625
:10398000AEADBFADE59718964D925D926D927C926B
:103990001B9749805A806B807C801C964D925D926B
:1039A0006D927C921F97FD01808A918AA28AB38AC8
:1039B00049845A846B847C8454964D925D926D92B6
:1039C0007C925797E3968EAD9FADE397CC58DF4F2F
:1039D0000FB6F894DEBF0FBECDBFDF91CF911F9120
:1039E0000F91FF90EF90DF90CF90BF90AF909F909E
:1039F0008F907F906F905F904F903F902F900895A1
:103A0000CF93DF93FC0181E093E2A5E4B7E68087E2
:103A10009187A287B38789E89BEAADECBFEE8487E4
:103A20009587A687B7878EEF9CEDAAEBB8E9808BC8
:103A3000918BA28BB38B86E794E5A2E3B0E1848BF4
:103A4000958BA68BB78B10821182128213821482FF
:103A5000158216821782DF01A85ABF4F80E4ED015C
:103A6000982F19929A95E9F77896DF011D928A9519
:103A7000E9F7DF91CF9108958F929F92AF92BF9215
:103A8000EF92FF920F931F93CF93DF93EC017B0193
:103A90008A0188819981AA81BB8160E070E04C0134
:103AA0005D01840E951EA61EB71E2FE1B2228882EC
:103AB0009982AA82BB8288169906AA06BB0668F478
:103AC0008C809D80AE80BF802FEF821A920AA20A5E
:103AD000B20A8C829D82AE82BF828F739927AA27F9
:103AE000BB270097A105B10531F120E4822E912C6E
:103AF000A12CB12C881A990AAA0ABB0A4896481523
:103B000059056A057B0528F4A801B7018C0F9D1F94
:103B100022C0A401B7018C0F9D1F0E94732CE80CDA
:103B2000F91C0819190940E450E0BE01685E7F4F96
:103B3000CE010E94810C0034110548F0A801407CA0
:103B4000B701CE010E94810C7C010F731127A801DF
:103B5000B701CE014896DF91CF911F910F91FF9051
:103B6000EF90BF90AF909F908F900C94732CEF923A
:103B7000FF920F931F93CF93DF938C01EB0148814A
:103B800059816A817B814F73552766277727DB012F
:103B9000CA010196A11DB11DFE01E40FF51F20E829
:103BA000208F40E450E060E070E0481B590B6A0B46
:103BB0007B0B9E01285E3F4F79014830510561051E
:103BC0007105A0F4489660E070E08C0F9D1F0E9484
:103BD0007C2C40E450E0B701CE010E94810C40E40F
:103BE00050E060E070E080E090E0DC014850510976
:103BF000489660E070E08C0F9D1F0E947C2C8881AD
:103C00009981AA81BB8123E0880F991FAA1FBB1F3E
:103C10002A95D1F788839983AA83BB83FE01E05B51
:103C2000FF4F8083319690833196A0833196B08385
:103C30003C812D819E818F81319630833196208306
:103C4000319690833196808340E450E0B701CE01F5
:103C50000E94810C8885F8018083898581838A850B
:103C600082838B8583838C8584838D8585838E85F4
:103C700086838F85878388898087898981878A89D8
:103C800082878B8983878C8984878D8985878E89B4
:103C900086878F89878788E9FE0111928A95E9F7DF
:103CA000DF91CF911F910F91FF90EF900895CF92E8
:103CB000DF92EF92FF920F931F93CF93DF93CDB7D5
:103CC000DEB7C859D1090FB6F894DEBF0FBECDBF1D
:103CD0007C016B0180E190E00E940D268C01CE01F9
:103CE00001960E94001DA601B701CE0101960E9417
:103CF0003C1DBE016F5F7F4FC8010E94B71DC80108
:103D0000C856DF4F0FB6F894DEBF0FBECDBFDF91B0
:103D1000CF911F910F91FF90EF90DF90CF9008957A
:103D2000CF93DF931F92CDB7DEB76983DC01ED91AE
:103D3000FC910280F381E02D41E050E0BE016F5F15
:103D40007F4F09950F90DF91CF9108950895FC0161
:103D50001382128288EE93E0A0E0B0E08483958322
:103D6000A683B7838FE291E09183808380E5848787
:103D700081E085878AE090E09787868789E090E0F8
:103D8000918B808B82E090E0938B828B148A158AD2
:103D9000168A178A118E108E138E128E158E148E1F
:103DA00040E050E0BA01CF010C943E25FC0177873A
:103DB0006687518B408B338B228B08950F931F9313
:103DC000CF93DF93EC01062F142F60E08E850E94C5
:103DD00098284C853D8580918C38882399F02FB7A1
:103DE000F89480918C38813059F48DB380938A385F
:103DF0009DB380918B38809589238DBB2FBF02C0E6
:103E000020938A384CBD3DBD0EBD00000DB407FEA9
:103E1000FDCF8EB51EBD00000DB407FEFDCF1EB553
:103E200080918C38882361F09FB7F89420918C386A
:103E300080918A38213019F48DBB9FBF01C08FBF9C
:103E400061E08E850E949828812FDF91CF911F918C
:103E50000F9108956F7740E00C94DE1E68E10C949A
:103E60002A1F0F931F93CF93DF938C016AE10E9467
:103E70002A1FC82FD0E0F80164897589868997893F
:103E80000E94292A24ED30E843E45EE40E94222ABD
:103E900087FD2797CE018D599109DF91CF911F9111
:103EA0000F910895CF93DF93EC0163E10E942A1FE5
:103EB00090E0288D398D821B930BDF91CF9108956F
:103EC000CF93DF93EC01E881F9810480F581E02D47
:103ED0000995892B59F0888D998D0196998F888F36
:103EE00060E0CE010E942A1F90E002C08FEF9FEF9A
:103EF000DF91CF9108950F931F93CF93DF938C01A0
:103F000066E00E942A1FD82F67E0C8010E942A1F7E
:103F1000C82F68E0C8010E942A1F4C2F50E060E0C3
:103F200070E0762F652F542F44276D2B8A019B015B
:103F3000082BC901B80120E038E448EE51E00E94A6
:103F4000F82A03E10E949D2BB901CA01DF91CF91AC
:103F50001F910F9108956DE10E942A1FE82FF0E054
:103F600084E0F595E7958A95E1F7EA30F105F8F4F4
:103F7000EA5BFF4F0C94DD2A60EA78E21EC060E441
:103F800071E51BC062E17AE718C064EE72EA15C001
:103F900064E274EF12C068E478EE81E00FC060E97B
:103FA00070ED83E00BC060E271EA87E007C008951E
:103FB00068E77EE102C060EF7CE380E090E0089576
:103FC0006CE20C942A1FCF93DF93EC0143E861E885
:103FD0000E94DE1E62E1CE010E942A1F83FD03C003
:103FE0000E94C728F7CF48E062E9CE010E94DE1E9A
:103FF00081E090E0DF91CF910895AF92BF92CF9290
:10400000DF92FF920F931F93CF93DF936C015B01BD
:10401000EA0162E20E942A1FF82E90E09C012C0F18
:104020003D1F2F3F310529F020F0CFEFD0E0C81B16
:10403000D90B8501AC0EBD1E0A151B0541F0F80118
:1040400041918F0160E8C6010E94DE1EF5CF4C2F22
:104050004F0D62EAC6010E94DE1ECE01DF91CF91B4
:104060001F910F91FF90DF90CF90BF90AF90089578
:104070000F931F93CF93DF93EC01E881F9810480C4
:10408000F581E02D0995892B91F06DE0CE010E941C
:104090002A1F082F60E0CE010E942A1F182F402FF0
:1040A0006DE8CE010E94DE1E812F90E002C08FEFEE
:1040B0009FEFDF91CF911F910F910895CF93DF93E1
:1040C000EC017D8F6C8F672BA9F160E08A890E94DB
:1040D0005C2840E060ECCE010E94DE1E8A899B894C
:1040E0008230910539F08A30910531F00B9731F02B
:1040F0008FEF05C082E003C080E001C081E00E9434
:104100009E238A899B898230910539F08A309105F6
:1041100031F00B9731F08FEF05C082E003C080E0F3
:1041200001C081E043E050E06DE273E2DF91CF91A6
:104130000C94C9288A899B898230910539F08A308C
:10414000910531F00B9731F08FEF05C082E003C08D
:1041500080E001C081E00E94F8288A899B89823032
:10416000910539F08A30910531F00B9731F08FEFDE
:1041700005C082E003C080E001C081E0DF91CF9103
:104180000C94BD2341E861E80C94DE1E40E861E830
:104190000C94DE1E0E94C6200C948A23AF92BF921C
:1041A000CF92DF92EF92FF920F931F93CF93DF9303
:1041B000EC01DB01CA014C8B5D8B6E8B7F8B6A013E
:1041C0007B01FF0CCC08DC2C76019A01AD016C2D33
:1041D0007C2D8C2D9C2D03E10E94822BA12CE8E4E8
:1041E000BE2EF8EECF2EDD24D394E12CF12C00E08E
:1041F00010E00E94252B122FC22ED32E7A01A70188
:104200006627772766E8CE010E94DE1E77276F2D8E
:104210005E2D4D2D67E8CE010E94DE1E412F68E81D
:10422000CE01DF91CF911F910F91FF90EF90DF9022
:10423000CF90BF90AF900C94DE1E0F931F93CF933F
:10424000DF938C01EB016630710534F06D30710540
:1042500084F46630710579F445EC61EBC8010E9485
:10426000DE1E4CE067EBC8010E94DE1EC6E0D0E017
:104270000CC0CCE0D0E043EC61EBC8010E94DE1E34
:104280004AE067EBC8010E94DE1E6EE1C8010E9491
:104290002A1F8F7094E0CC0FDD1F9A95E1F74C2F09
:1042A000482B6EE9C801DF91CF911F910F910C94BB
:1042B000DE1ECF92DF92EF92FF920F931F93CF9368
:1042C000DF938C01CB01BA010E94292A6B017C018A
:1042D00020E030EC43EF55E40E94222A18160CF03F
:1042E00056C020E030E842E256E4C701B6010E9421
:1042F000222A18160CF04EC020E030EC43E756E4BA
:10430000C701B6010E94222A18160CF046C020E010
:1043100030E842EA56E4C701B6010E94222A181684
:104320000CF03EC020E034E244EF56E4C701B60191
:104330000E94222A1816BCF520E034EE42E257E42F
:10434000C701B6010E94222A181684F520E034E243
:1043500044E757E4C701B6010E94222A18164CF51B
:1043600020E034E244EF57E4C701B6010E94222A5C
:10437000181614F520E034E244E758E4C701B6010A
:104380000E94222A1816DCF4C9E0D0E01AC0C0E06E
:10439000D0E017C0C1E0D0E014C0C2E0D0E011C04E
:1043A000C3E0D0E00EC0C4E0D0E00BC0C5E0D0E078
:1043B00008C0C6E0D0E005C0C7E0D0E002C0C8E059
:1043C000D0E06DE1C8010E942A1F8F7094E0CC0FED
:1043D000DD1F9A95E1F74C2F482B6DE9C801DF915D
:1043E000CF911F910F91FF90EF90DF90CF900C94A1
:1043F000DE1E0F931F93CF93DF938C016530710501
:104400003CF0EB01693071052CF0C8E0D0E002C04F
:10441000C5E0D0E06DE1C8010E942A1F2497CC0FAF
:10442000DD1F817F4C2F482B6DE9C801DF91CF91B3
:104430001F910F910C94DE1ECF93DF93EC016EE180
:104440000E942A1F482F44606EE9CE01DF91CF9170
:104450000C94DE1ECF93DF93EC011B8E1A8E6DE160
:104460000E942A1F482F4E7F6DE9CE01DF91CF9128
:104470000C94DE1ECF93DF93EC0181E090E09B8FE4
:104480008A8F6DE1CE010E942A1F482F41606DE99D
:10449000CE01DF91CF910C94DE1E0F931F93CF932B
:1044A000DF93EC018B010E94C220CE01012B19F099
:1044B0000E943A2202C00E942A2240E06DE8CE010A
:1044C0000E94DE1E40E062EACE010E94DE1E81E014
:1044D00090E0DF91CF911F910F9108950F931F935B
:1044E000CF93DF93EC018B011616170644F40E945C
:1044F0003A22402F62EACE010E94DE1E02C00E94D4
:104500002A2245E861E8CE01DF91CF911F910F91FA
:104510000C94DE1ECF92DF92EF92FF92CF93DF9347
:10452000EC016A017B0161E08E850E945C2861E0FC
:104530008E850E949828888999898F3F2FEF92074E
:10454000B9F061E00E945C2860E088890E949828A8
:104550006AE070E080E090E00E94A92761E088892D
:104560000E9498286AE070E080E090E00E94A9270D
:104570000E94542362E4CE010E942A1F823161F519
:10458000CE010E94C620B701A601CE010E94CE2016
:1045900040E06EE8CE010E94DE1E40E06FE8CE01F2
:1045A0000E94DE1E6CE0CE010E942A1F482F43604D
:1045B0006CE8CE010E94DE1E44E066EACE010E9455
:1045C000DE1E40E869E8CE010E94DE1ECE010E9498
:1045D000C22081E090E002C080E090E0DF91CF91C6
:1045E000FF90EF90DF90CF9008951F93CF93DF93CC
:1045F000EC0162E10E942A1F182F482F62E9CE01C8
:104600000E94DE1E15FD25C0198E188E8A8D9B8D89
:10461000892B11F062E201C063E1CE010E942A1FE2
:10462000182F60E1CE010E942A1F482F6DE8CE01AD
:104630000E94DE1EEC8DFD8D309719F0812F90E0E9
:10464000099540E06DE8CE01DF91CF911F910C9468
:10465000DE1EDF91CF911F9108958CE698E30C94B4
:10466000F522452B61F46F30710514F06EE070E0B7
:1046700077FF02C060E070E0462F40670EC06230F6
:10468000710534F0623171052CF061E170E002C017
:1046900062E070E06250462F406869E80C94DE1ECC
:1046A0008CE698E30C94A71ECF93CFB7F894809133
:1046B0008D38811127C0ECE0F1E08491ECEEF0E060
:1046C0009491E82FF0E0EE0FFF1FEE5CFE4FA591F6
:1046D000B491EC91E92321F461E084E00E949828F0
:1046E00061E084E00E945C288CB580618CBD8CB553
:1046F00080648CBD61E087E00E945C2861E085E019
:104700000E945C2880918D388F5F80938D38CFBF59
:10471000CF9108959FB7F89480918D38882319F030
:10472000815080938D3880918D38811105C08CB572
:104730008F7B8CBD10928C389FBF08959FB7F894E3
:10474000813029F058F0823021F484E008C082E002
:1047500006C082E080938C3880E001C081E0209127
:104760008B38822B80938B3880918C38811103C0D9
:1047700081E080938C389FBF089590918C3892305F
:10478000B1F02FB7F894833030F4E82FF0E0E55C17
:10479000FE4F808101C080E0809590918B38892305
:1047A00080938B38811102C010928C382FBF0895EE
:1047B000CF92DF92EF92FF920F931F93CF93DF93ED
:1047C0006C017A018B01C0E0D0E0CE15DF0581F0ED
:1047D000D8016D918D01D601ED91FC910190F08190
:1047E000E02DC6010995892B11F02196EECF7E01AF
:1047F000C701DF91CF911F910F91FF90EF90DF9054
:10480000CF900895FC01918D228D892F90E0805CDE
:104810009F4F821B91098F7399270895FC01918DF9
:10482000828D981731F0828DE80FF11D858D90E013
:1048300008958FEF9FEF0895FC01918D828D981759
:1048400061F0828DDF01A80FB11D5D968C91928D74
:104850009F5F9F73928F90E008958FEF9FEF089571
:1048600084EA95E2892B41F080E090E0892B21F0E9
:104870000E94A42581110DC080E090E0892B71F089
:1048800080E090E0892B51F00E940000811104C06B
:1048900008950E940000F0CF0C9400000895FC01E0
:1048A000848DDF01A80FB11DA35ABF4F2C91848DB9
:1048B00090E001968F739927848FA689B7892C93EE
:1048C000A089B1898C9180648C93938D848D981389
:1048D00006C00288F389E02D80818F7D8083089552
:1048E000EF92FF920F931F93CF93DF93EC0181E040
:1048F000888F9B8D8C8D981305C0E889F9898081FC
:1049000085FD24C0F62E0B8D10E00F5F1F4F0F7337
:104910001127E02E8C8DE8120CC00FB607FCFACFE1
:10492000E889F989808185FFF5CFCE010E944F2467
:10493000F1CF8B8DFE01E80FF11DE35AFF4FF0829E
:104940000B8FEA89FB898081806207C0EE89FF892D
:104950006083E889F98980818064808381E090E0C8
:10496000DF91CF911F910F91FF90EF900895CF931A
:10497000DF93EC01888D8823C9F0EA89FB89808167
:1049800085FD05C0A889B9898C9186FD0FC00FB639
:1049900007FCF5CF808185FFF2CFA889B9898C917A
:1049A00085FFEDCFCE010E944F24E7CFDF91CF915D
:1049B0000895CF92DF92EF92FF921F93CF93DF93F0
:1049C000EC016A017B01122FE889F98982E080837A
:1049D0004115514E61057105B1F060E079E08DE35C
:1049E00090E0A70196010E949C2ADA01C901019773
:1049F000A109B109B695A795979587959C012115B1
:104A000080E13807A8F0E889F989108260E874E845
:104A10008EE190E0A70196010E949C2ADA01C9016B
:104A20000197A109B109B695A795979587959C011E
:104A3000EC85FD853083EE85FF852083188EEC891B
:104A4000FD891083EA89FB89808180618083EA89FE
:104A5000FB89808188608083EA89FB898081806806
:104A60008083EA89FB8980818F7D8083DF91CF916C
:104A70001F91FF90EF90DF90CF900895FC01448349
:104A800055836683778308951F920F920FB60F9216
:104A900011240BB60F922F938F939F93EF93FF9355
:104AA000E0919E38F0919F388081E091A438F09198
:104AB000A53882FD12C090818091A7388F5F8F73D7
:104AC0002091A838821751F0E091A738F0E0E25722
:104AD000F74C958F8093A73801C08081FF91EF91AB
:104AE0009F918F912F910F900BBE0F900FBE0F9043
:104AF0001F9018951F920F920FB60F9211240BB6AC
:104B00000F922F933F934F935F936F937F938F9366
:104B10009F93AF93BF93EF93FF938EE898E30E9428
:104B20004F24FF91EF91BF91AF919F918F917F9112
:104B30006F915F914F913F912F910F900BBE0F900E
:104B40000FBE0F901F9018958EE898E30E940224E4
:104B500021E0892B09F420E0822F0895EEE8F8E3A4
:104B60001382128288EE93E0A0E0B0E08483958304
:104B7000A683B78382E491E09183808385EC90E003
:104B80009587848784EC90E09787868780EC90E017
:104B9000918B808B81EC90E0938B828B82EC90E008
:104BA000958B848B86EC90E0978B868B118E128E82
:104BB000138E148E089508950E94E5270E94DB2528
:104BC0000E942E07C0E3D4E20E94FC0B2097E1F381
:104BD0000E943024F9CF009729F0BC0180E090E0DA
:104BE0000C946A2C0895CF92DF92EF92FF92611598
:104BF00071058105910549F06B017C010E941C2C17
:104C0000A70196010E94BE2A03C060E070E0CB01BC
:104C1000FF90EF90DF90CF9008950F931F93CF9365
:104C2000DF938230910510F482E090E0E091363914
:104C3000F091373920E030E0A0E0B0E0309719F192
:104C4000408151810281138148175907C8F08417A8
:104C5000950769F4109731F012960C9312971396FA
:104C60001C9327C0009336391093373922C0211581
:104C7000310519F04217530718F49A01BD01EF01ED
:104C8000DF01F801DBCF21153105F9F0281B390BC5
:104C90002430310580F48A819B816115710521F0F2
:104CA000FB019383828304C0909337398093363914
:104CB000FE01329644C0FE01E20FF31F81939193EF
:104CC00022503109398328833AC0209134393091F8
:104CD0003539232B41F4209120013091210130936B
:104CE00035392093343920911E0130911F0121154F
:104CF000310541F42DB73EB7409122015091230177
:104D0000241B350BE0913439F0913539E217F30764
:104D1000A0F42E1B3F0B2817390778F0AC014E5F2B
:104D20005F4F2417350748F04E0F5F1F50933539FA
:104D3000409334398193919302C0E0E0F0E0CF01D9
:104D4000DF91CF911F910F910895CF93DF9300973B
:104D500009F481C0FC01329713821282A091363986
:104D6000B0913739109781F420813181820F931FE0
:104D700020913439309135392817390751F5F0939E
:104D80003539E093343967C0ED0120E030E0CE17CB
:104D9000DF0740F44A815B819E0141155105F1F026
:104DA000EA01F5CFD383C28340815181840F951FDF
:104DB000C817D90759F488819981840F951F0296E5
:104DC000918380838A819B8193838283211531051E
:104DD00029F4F0933739E09336393DC0E901FB837C
:104DE000EA8349915991C40FD51FEC17FD0761F46F
:104DF00080819181840F951F0296E90199838883B0
:104E0000828193819B838A83E0E0F0E012968D910A
:104E10009C911397009719F0FD01DC01F7CF8D915C
:104E20009C9111979D012E5F3F4F820F931F209100
:104E30003439309135392817390769F4309729F416
:104E4000109237391092363902C013821282B09311
:104E50003539A0933439DF91CF9108951F920F9285
:104E60000FB60F9211242F933F938F939F93AF937D
:104E7000BF9380912C3990912D39A0912E39B0910A
:104E80002F3930912B3923E0230F2D3720F4019651
:104E9000A11DB11D05C026E8230F0296A11DB11D5D
:104EA00020932B3980932C3990932D39A0932E3950
:104EB000B0932F398091303990913139A0913239A6
:104EC000B09133390196A11DB11D80933039909373
:104ED0003139A0933239B0933339BF91AF919F915B
:104EE0008F913F912F910F900FBE0F901F901895AB
:104EF0002FB7F89460912C3970912D3980912E390B
:104F000090912F392FBF08953FB7F8948091303991
:104F100090913139A0913239B091333926B5A89B9F
:104F200005C02F3F19F00196A11DB11D3FBFBA2F3B
:104F3000A92F982F8827820F911DA11DB11DBC019B
:104F4000CD0142E0660F771F881F991F4A95D1F760
:104F500008958F929F92AF92BF92CF92DF92EF927D
:104F6000FF926B017C010E9484274B015C01C114FC
:104F7000D104E104F10401F10E94C7280E948427B2
:104F8000DC01CB0188199909AA09BB09883E934025
:104F9000A105B10560F321E0C21AD108E108F108CA
:104FA00088EE880E83E0981EA11CB11CC114D104A8
:104FB000E104F10419F7DBCFFF90EF90DF90CF9081
:104FC000BF90AF909F908F900895789484B5826041
:104FD00084BD84B5816084BD85B5826085BD85B59D
:104FE000816085BDEEE6F0E0808181608083E1E84C
:104FF000F0E0108280818260808380818160808384
:10500000E0E8F0E0808181608083E1EBF0E0808186
:1050100084608083E0EBF0E0808181608083E1E95F
:10502000F0E0808182608083808181608083E0E91C
:10503000F0E0808181608083EAE7F0E08081846035
:105040008083808182608083808181608083808191
:10505000806880831092C100089590E0FC01319730
:10506000EA30F10540F5E05BFF4F0C94DD2A8091BA
:1050700080008F7703C0809180008F7D80938000B7
:10508000089584B58F7702C084B58F7D84BD08955F
:105090008091B0008F7703C08091B0008F7D8093A6
:1050A000B0000895809190008F7703C080919000A8
:1050B0008F7D809390000895CF93DF9390E0FC0163
:1050C000E851FF4F2491FC01E85FFE4F8491882353
:1050D00061F190E0880F991FFC01EE5CFE4FC591D5
:1050E000D491FC01E85DFE4FA591B491611109C016
:1050F0009FB7F8948881209582238883EC912E2392
:105100000BC0623061F49FB7F8948881322F3095DC
:1051100083238883EC912E2B2C939FBF06C08FB7DF
:10512000F894E8812E2B28838FBFDF91CF910895CB
:105130001F93CF93DF93282F30E0F901E853FF4FFF
:105140008491F901E851FF4FD491F901E85FFE4FD6
:10515000C491CC23C1F0162F81110E942D28EC2F71
:10516000F0E0EE0FFF1FE85DFE4FA591B4919FB7F1
:10517000F894111104C08C91D095D82302C0EC9101
:10518000DE2BDC939FBFDF91CF911F91089508958F
:105190000895833060F5E82FF0E0EE0FFF1FEC5D1F
:1051A000FE4F71836083813051F08230A1F0809195
:1051B00069008C7F482B40936900E89A089580919C
:1051C0006900837F440F551F440F551F482B4093A0
:1051D0006900E99A0895809169008F7C94E0440FFA
:1051E000551F9A95E1F7482B40936900EA9A089574
:1051F000833098F4813021F0823021F0E89803C0A8
:10520000E99801C0EA98E82FF0E0EE0FFF1FEC5D8F
:10521000FE4F88EC98E29183808308951F920F924D
:105220000FB60F9211240BB60F922F933F934F930B
:105230005F936F937F938F939F93AF93BF93EF93FE
:10524000FF93E0912401F09125010995FF91EF91E1
:10525000BF91AF919F918F917F916F915F914F918E
:105260003F912F910F900BBE0F900FBE0F901F908C
:1052700018951F920F920FB60F9211240BB60F9232
:105280002F933F934F935F936F937F938F939F934E
:10529000AF93BF93EF93FF93E0912601F091270125
:1052A0000995FF91EF91BF91AF919F918F917F9160
:1052B0006F915F914F913F912F910F900BBE0F9087
:1052C0000FBE0F901F9018951F920F920FB60F925E
:1052D00011240BB60F922F933F934F935F936F93CD
:1052E0007F938F939F93AF93BF93EF93FF93E0913F
:1052F0002801F09129010995FF91EF91BF91AF919C
:105300009F918F917F916F915F914F913F912F91DD
:105310000F900BBE0F900FBE0F901F901895883006
:1053200028F0883110F0885101C08FEF20912A01B8
:1053300090E4299F900111248770822B80937C0038
:1053400080917A00806480937A0080917A0086FD53
:10535000FCCF809178002091790090E0922B089505
:105360001F93CF93DF93182FEB0161E00E945C281D
:10537000209711F460E004C0CF3FD10539F461E01B
:10538000812FDF91CF911F910C949828E12FF0E0AD
:10539000E853FF4FE4918E2F90E0FC013197EA3003
:1053A000F10508F046C0E65AFF4F0C94DD2A84B59B
:1053B000806884BDC7BD42C084B5806284BDC8BD5D
:1053C0003DC080918000806880938000D0938900E8
:1053D000C093880033C080918000806280938000F9
:1053E000D0938B00C0938A0029C08091B000806860
:1053F0008093B000C093B30021C08091B000806260
:105400008093B000C093B40019C080919000806870
:1054100080939000D0939900C09398000FC0809122
:105420009000806280939000D0939B00C0939A007C
:1054300005C0C038D1050CF0A2CF9CCFDF91CF9131
:105440001F9108950E94642A08F481E00895E89469
:1054500009C097FB3EF490958095709561957F4FBC
:105460008F4F9F4F9923A9F0F92F96E9BB2793956A
:10547000F695879577956795B795F111F8CFFAF47A
:10548000BB0F11F460FF1BC06F5F7F4F8F4F9F4FAB
:1054900016C0882311F096E911C0772321F09EE809
:1054A000872F762F05C0662371F096E8862F70E06F
:1054B00060E02AF09A95660F771F881FDAF7880F49
:1054C0009695879597F90895990F0008550FAA0B9F
:1054D000E0E8FEEF16161706E807F907C0F0121607
:1054E0001306E407F50798F0621B730B840B950B0A
:1054F00039F40A2661F0232B242B252B21F408955F
:105500000A2609F4A140A6958FEF811D811D0895FB
:10551000AA1BBB1B51E107C0AA1FBB1FA617B707D9
:1055200010F0A61BB70B881F991F5A95A9F78095F5
:105530009095BC01CD010895A1E21A2EAA1BBB1BB8
:10554000FD010DC0AA1FBB1FEE1FFF1FA217B3074F
:10555000E407F50720F0A21BB30BE40BF50B661F65
:10556000771F881F991F1A9469F760957095809529
:1055700090959B01AC01BD01CF010895052E97FBCD
:105580001EF400940E94D52A57FD07D00E949C2A41
:1055900007FC03D04EF40C94D52A509540953095D5
:1055A00021953F4F4F4F5F4F08959095809570958F
:1055B00061957F4F8F4F9F4F0895EE0FFF1F00247F
:1055C000001C0BBE0790F691E02D099469279627E1
:1055D000692778278727782708950E94B92BA59FE8
:1055E000900DB49F900DA49F800D911D11240895DE
:1055F000E894DF93CF93FC01DB010E94B92B7F93EA
:105600006F93E9019A01AC01BF93AF933F932F933E
:10561000DF010E94B92B26F46C1B7D0B820B930BD0
:105620009E01EB01FC010E94C82BAF91BF912F910D
:105630003F910E94C82BBE01CF01F9012F913F91EC
:10564000CF91DF910895689401C0E8948F929F9262
:10565000CF93DF930E94312BDF91CF919F908F905A
:10566000089588249924F401E401B0E49F93AA27C3
:105670009A158B049C04ED05FE05CF05D007A10704
:1056800098F4AD2FDC2FCF2FFE2FE92D982C892EEB
:10569000982F872F762F652F542F432F322F2227B5
:1056A000B85031F7BF9127C01B2EBF91BB27220FE7
:1056B000331F441F551F661F771F881F991F881CA3
:1056C000991CEE1FFF1FCC1FDD1FAA1FBB1F8A14D2
:1056D0009B04EC05FD05CE05DF05A007B10748F0EA
:1056E0008A189B08EC09FD09CE09DF09A00BB10B54
:1056F00021601A94E1F62EF49401AF01BE01CD01B0
:10570000000C08950F93083090F0982F872F762F74
:10571000652F542F432F322F22270850F4CF220F0A
:10572000331F441F551F661F771F881F991F0A9537
:10573000B2F70F91089597FB10F8169400080F9395
:10574000083098F00850232F342F452F562F672FFD
:10575000782F892F902DF4CF05949795879577957D
:10576000679557954795379527950A95AAF70F910D
:105770000895A29FB001B39FC001A39F700D811D2A
:105780001124911DB29F700D811D1124911D08954A
:105790000E94B92B460F571FC81FD91F08F4319616
:1057A00008958F929F92AF92BF92CF92DF92EF9225
:1057B000FF92CF93DF93EC01688179818A819B818D
:1057C000611571058105910521F464E279ED8BE5A0
:1057D00097E02DE133EF41E050E00E94BE2A4901FD
:1057E0005A019B01AC01A7EAB1E40E94ED2A6B01CA
:1057F0007C01ACEEB4EFA50194010E949C2CDC016D
:10580000CB018C0D9D1DAE1DBF1DB7FF03C00197C1
:10581000A109B04888839983AA83BB83BC01CD01C9
:105820009F77DF91CF91FF90EF90DF90CF90BF9067
:10583000AF909F908F9008958F929F92AF92BF925A
:10584000CF92DF92EF92FF9260910001709101017F
:105850008091020190910301611571058105910507
:1058600021F464E279ED8BE597E02DE133EF41E03F
:1058700050E00E94BE2A49015A019B01AC01A7EAEF
:10588000B1E40E94ED2A6B017C01ACEEB4EFA501FE
:1058900094010E949C2CDC01CB018C0D9D1DAE1D42
:1058A000BF1DB7FF03C00197A109B0488093000155
:1058B00090930101A0930201B0930301BC01CD01BB
:1058C0009F77FF90EF90DF90CF90BF90AF909F9029
:1058D0008F900895609300017093010180930201FD
:1058E000909303010895FB01DC0102C001900D9229
:1058F00041505040D8F70895DC0101C06D934150EC
:105900005040E0F70895F999FECF92BD81BDF89A15
:10591000992780B50895262FF999FECF1FBA92BD19
:1059200081BD20BD0FB6F894FA9AF99A0FBE019680
:105930000895B7FF0C94ED2A0E94ED2A821B930B69
:065940000895F894FFCF6A
:1059460001000000F82A000028013C000000FE03C8
:105956000000000F00FFDCFE1101FF000500000043
:1059660038398000C828C828C828010000000090DF
:105976001EFD1F521F601F3820A61E0102040000D4
:0E59860000007024D82302241C240E24B72411
:00000001FF
